:040000008131DB2946
:10000800803120007F08F4000B1DC0290B11181047
:100018001708FA001608F9007D08031D78287B08E0
:100028007C04031D1B287A08FC007908FB007B0E62
:100038000F39F5007C0EF039F5047C0E0F39F60007
:100048007C08F1007B08F0000730F136F00C890BD2
:1000580029287008F7007108F8007509F00076097A
:10006800F100F00A0319F10A7B087007F2007C0816
:10007800713DF30073087A02031D4428720879025F
:10008800031848288D1678287709F0007809F100B8
:10009800F00A0319F10A7B087007F2007C08713D29
:1000A800F3007A087302031D5B28790872020318AB
:1000B800772877087B07F00078087C3DF100710805
:1000C8007A02031D692870087902031877287908CD
:1000D8007B07F0007A087C3DF100F136F00C7008DF
:1000E800FB007108FC008D127D03031DE028200829
:1000F8002104031D83287A08A1007908A000200E96
:100108000F39F500210EF039F504210E0F39F600EC
:100118002108F1002008F0000730F136F00C890BB7
:1001280091287008F7007108F8007509F000760941
:10013800F100F00A0319F10A20087007F2002108FB
:10014800713DF30073087A02031DAC287208790226
:100158000318B0280D16E0287709F0007809F10097
:10016800F00A0319F10A20087007F2002108713D0E
:10017800F3007A087302031DC32879087202031872
:10018800DF2877082007F0007808213DF100710882
:100198007A02031DD128700879020318DF2879082C
:1001A8002007F0007A08213DF100F136F00C7008C4
:1001B800A0007108A1000D1202307D06031D492917
:1001C80022082304031DEC287A08A3007908A2005A
:1001D800220E0F39F500230EF039F504230E0F39DE
:1001E800F6002308F1002208F0000730F136F00C81
:1001F800890BFA287008F7007108F8007509F000F3
:100208007609F100F00A0319F10A22087007F200D2
:100218002308713DF30073087A02031D152972083B
:100228007902031819298D1549297709F0007809E9
:10023800F100F00A0319F10A22087007F2002308F6
:10024800713DF3007A087302031D2C2979087202A4
:100258000318482977082207F0007808233DF100A1
:1002680071087A02031D3A2970087902031848298F
:1002780079082207F0007A08233DF100F136F00CE6
:100288007008A2007108A3008D1103307D06031DBC
:10029800B22924082504031D55297A08A5007908E0
:1002A800A400240E0F39F500250EF039F504250EAB
:1002B8000F39F6002508F1002408F0000730F13660
:1002C800F00C890B63297008F7007108F8007509AC
:1002D800F0007609F100F00A0319F10A2408700702
:1002E800F2002508713DF30073087A02031D7E2988
:1002F80072087902031882290D15B2297709F000CE
:100308007809F100F00A0319F10A24087007F200CD
:100318002508713DF3007A087302031D95297908B1
:1003280072020318B12977082407F0007808253DE0
:10033800F10071087A02031DA329700879020318D5
:10034800B12979082407F0007A08253DF100F13633
:10035800F00C7008A4007108A5000D110130F00020
:100368007008FD0704307D020318FD017D089F0019
:100378009601970195011814911CD8299110013004
:10038800A7022708031DD0297D30F0007008A700B8
:100398000430F0007008A60026080319D729013098
:1003A800A6020D14D8290D107408FF000900813128
:1003B800DD29FB01FC01FD01A001A101A201A301AE
:1003C800A401A501A60120008131EA298B012100A1
:1003D800910192019301940120008C0122008C016B
:1003E8000F3023008C000F3021008C0020008D017D
:1003F80022008D0123008D0121008D017D30200018
:10040800A8002808A700A601FD01FB01FC01A00126
:10041800A101A201A301A401A5010B178B162100BC
:1004280091140C3020009E007D089F00C3302100ED
:100438009500C4302000980039309C00FA309B00A9
:100448009E17960197019A01950118141C158B1790
:020458002C2A4C
:020000040001F9
:04000E00C1CFFFD887
:00000001FF
